:106649000A2A2A2A2A2A2A2A2A2A2A2A2A2A2A2AC1
:106659002A2A20CFE0F0E0ECE5F2F0FB20E0E4E0CC
:10666900EFF2E5F0E0202A2A2A2A2A2A2A2A2A2AC7
:106679002A2A2A2A2A2A2A2A0A00312E204D414367
:1066890020E0E4F0E5F13A20200025303262783A42
:106699000008200A00322E20495020E0E4F0E5F1FC
:1066A9003A202020002562752E00332E20D8EBFEDB
:1066B900E73A2020202020202000342E20CCE0F1B1
:1066C900EAE020F1E5F2E83A2000352E2049502091
:1066D900E0E4F0E5F120F1E5F0E2E5F0E0313A201F
:1066E90000362E20495020E0E4F0E5F120F1E5F0F4
:1066F900E2E5F0E0323A2000372E20CFEEF0F2202A
:10670900EAEEEDF4E8E3F3F0E0F6E8E83A2025757F
:106719000A00382E20CFEEF0F220E4E0EDEDFBF593
:106729003A2020202020202025750A00392E20D249
:10673900E0E9EC2DE0F3F220EEF2E2E5F2E020F1FF
:10674900E5F0E2E5F0E03A202562752028312F31A5
:1067590030736563290A00302E20D1F2F0EEEAE0A9
:1067690020EAEEEDF43A202573200A00C7C0CFC80D
:10677900D1DC20466C61736820CFC0CCDFD2C82041
:106789000020C7E0EFE8F1FC20E7E0E2E5F0F8E5FA
:10679900EDE020210A000A53696E636F6D495020AC
:1067A9005665722E20312E32204343202827502748
:1067B9002DE2F5EEE420E220EAEEEDF4E8E3F3F071
:1067C900E0F2EEF029000A3E20CAEEEDF4E8E3F328
:1067D900F0E0F6E8EEEDEDFBE920F0E5E6E8EC0A9D
:1067E9000A00203C493E20203A20CFEEEAE0E7E0CB
:1067F900F2FC20EFE0F0E0ECE5F2F0FB0A00203CCF
:10680900536E3E203A20C7E0E4E0F2FC20EFE0F0CE
:10681900E0ECE5F2F020276E270A00203C4B3E20F1
:10682900203A20C7E0E4E0F2FC20EAEBFEF720E49E
:10683900EEF1F2F3EFE00A00203C573E20203A2027
:10684900C7E0EFE8F1E0F2FC20E8E7ECE5EDE5ED83
:10685900E8FF0A00203C4C3E20203A20C7E0E3F044
:10686900F3E7E8F2FC20EFF0EEE3F0E0ECECF30AFA
:1068790000203C453E20203A20C2FBF5EEE40A0008
:106889003E20C2E2E5E4E8F2E520EAEEECE0EDE4E0
:10689900F33A20000A00C2E2E5E4E8F2E520274DD8
:1068A900414320E0E4F0E5F15B2562645D273A208D
:1068B900256278202D3E0025627800C2E2E5E4E8F1
:1068C900F2E52027495020E0E4E0EFF2E5F0E05B53
:1068D9002562645D273A20256275202D3E002562D8
:1068E9007500C2E2E5E4E8F2E52027D8EBFEE75BB4
:1068F9002562645D273A20256275202D3E00C2E29B
:10690900E5E4E8F2E52027CCE0F1EAF3D1E5F2E8A5
:106919005B2562645D273A20256275202D3E00C201
:10692900E2E5E4E8F2E52027495020F1E5F0E2E567
:10693900F0E0315B2562645D273A20256275202DE0
:106949003E00C2E2E5E4E8F2E52027495020F1E5FE
:10695900F0E2E5F0E0325B2562645D273A202562CA
:1069690075202D3E000AC2E2E5E4E8F2E52027CFD2
:10697900EEF0F220EAEEEDF4E8E3F3F0E0F6E8E811
:10698900273A202575202D3E002575000AC2E2E52B
:10699900E4E8F2E52027CFEEF0F220E4E0EDEDFBAC
:1069A900F5273A202575202D3E000AC2E2E5E4E8E4
:1069B900F2E52027C2F0E5ECFF20EEE6E8E4E0EDA1
:1069C900E8FF20EEF2E2E5F2E0273A2025627520A1
:1069D9002D3E000AC2E2E5E4E8F2E52027F1F2F0F3
:1069E900EEEAF320EAEEEDF4E8E3F3F0E0F6E8E8A6
:1069F900273A0A2D3E00082008000A204572726FC6
:106A090072210A000AC2E2E5E4E8F2E520EAEBFEB7
:106A1900F720E4EEF1F2F3EFE03A0A2D3E000AC85E
:106A2900C4C5D220C7C0CFC8D1DC2120C6C4C8D2B2
:106A3900C521000AC7C0CFC8D1DC20C7C0C2C5D094
:106A4900D8C5CDC0210A000AC2E2E5E4E8F2E52092
:106A5900F0E0E7ECE5F020F4E0E9EBE0203E3E2051
:106A6900000ACA20EFF0E8E5ECF320E3EEF2EEE2EB
:106A7900210A000AD4E0E9EB20EFEEEBF3F7E5EDAC
:036A8900210A00DF
:10754400C2ADE4F5C9D2CDD2CCC2C9C2CAF5CDF51B
:10755400CC75CBFF75CAB885CBCD85CACCD29ED2AB
:107564009CD2CAE59924FF92CAC2ACC298C299308F
:0675740099032098FA22A1
:077664003098FDAF99C298B8
:01766B0022FC
:06764A00127664EFF52248
:087650008F993099FDC29922C7
:1075AE00E4FDFCC3ED9FEC9E5014E4FBFA0BBB0014
:0E75BE00010AEBF44A70F60DBD00010C80E5E9
:0175CC00229C
:047501008E2D8F2E0E
:10750500E4FBFAF52FF530C3E530952EE52F952DE3
:10751500502C1276648B828A83EFF0AE2FAF307CCD
:10752500017DF412728DED4C70057F2A127650059F
:0E75350030E5307002052F0BBB00010A80C943
:017543002225
:07766C003098FDAF99C298B0
:0176730022F4
:10763A00AE07BE0A057F0D127650AF0612765022AB
:1070FF007BFF7A667949126AEE7BFF7A6679831293
:10710F006AEEE4F52B7BFF7A667993748C252BF569
:10711F0082E43460F583E0F539126AEE052BE52B36
:10712F00C3940640E07BFF7A66799A126AEE7BFF82
:10713F007A66799E126AEEE4F52B7BFF7A6679AE5A
:10714F007492252BF582E43460F583E0F539126AE9
:10715F00EE052BE52BC3940440E07BFF7A66799A0A
:10716F00126AEE7BFF7A6679B3126AEEE4F52B7B37
:10717F00FF7A6679AE7484252BF582E43460F5834B
:10718F00E0F539126AEE052BE52BC3940440E07B42
:10719F00FF7A66799A126AEE7BFF7A6679C3126A72
:1071AF00EEE4F52B7BFF7A6679AE7488252BF5829A
:1071BF00E43460F583E0F539126AEE052BE52BC355
:1071CF00940440E07BFF7A66799A126AEE7BFF7A2D
:1071DF006679D3126AEEE4F52B7BFF7A6679AE748B
:1071EF009B252BF582E43460F583E0F539126AEEC6
:1071FF00052BE52BC3940440E07BFF7A66799A1246
:10720F006AEE7BFF7A6679EA126AEEE4F52B7BFF72
:10721F007A6679AE749F252BF582E43460F583E0AE
:10722F00F539126AEE052BE52BC3940440E07BFF82
:10723F007A66799A126AEE7BFF7A67790190609984
:10724F00E0F539A3E0F53A126AEE7BFF7A67791B16
:10725F00906097E0F539A3E0F53A126AEE7BFF7A7A
:10726F006779359060A3E0F539126AEE75390175CB
:0E727F003A60753B007BFF7A677960026AEE29
:0673FA008E2D8F2E8D2F59
:10740000E4F534F535F532F533E52F60097BFF7A85
:10741000677975126AEEE4F530F531E52DC4F8545C
:10742000F0C868FEE52EC4540F48FFC3E5319FE560
:10743000309E5042AE34AF35AD07AC067B10AF3353
:10744000AE3212757A74102535F535E43534F534DD
:1074500074102533F533E43532F532E52F600DE550
:1074600031541F7007FBFA7923126AEE0531E531BA
:1074700070A9053080A5E52DC4F854F0C868FEE574
:107480002EC4540F48C4F8540FC868FFEEC454F01B
:1074900048FEC3E52E9FFFE52D9EAC34AD35AB070E
:1074A000AF33AE3212757AE52F60097BFF7A6779C8
:0474B0008A126AEEE4
:0174B40022B5
:10600300752501C2AF907FFEE0B4FF047F018002DB
:106013007F00907FFDE0B4AA047E0180027E00EE43
:106023005FFF907FFFE0B455047E0180027E00EEA7
:106033005F6028E4907FFDF0A3F0A3F0907FF0E091
:10604300FEA3E0FF4E6005E4FD1273FA7BFF7A00C6
:1060530079008B288A29892A127308127544C298F9
:106063007BFF7A67799F126AEE30980F7BFF7A0085
:1060730079008B288A29892A127308E4F523E4F529
:1060830024209803026614127664EFF522645060AC
:1060930009E52264706003026605AF221276507F21
:1060A3000A127650E4F523E52304FF1275CD7484B8
:1060B3002523F582E43460F583EFF00523E523C35C
:1060C300943F40E3E4F523E523247FFF1275CD7469
:1060D300002523F582E43460F583EFF00523E523FF
:1060E300C3948040E2E490607FF0E525700302668C
:1060F300147BFF7A6779CF126AEE7BFF7A6779EBBD
:10610300126AEE7BFF7A687907126AEE7BFF7A6880
:106113007924126AEE7BFF7A687941126AEE7BFF7B
:106123007A68795D126AEE7BFF7A68797A126AEE91
:106133007BFF7A687989126AEE12764AE522127237
:10614300E265A34561694964F64B65FF4C616F5392
:1061530065A95765A36561696965FF6C616F7365BF
:10616300A977000060ED1270FF0260ED12764AE538
:10617300221272E264793061993161F432624F33F1
:1061830062AA3463053563603663BB3763F93864E9
:106193003F39000064ED7BFF7A68799D126AEEE473
:1061A300F522E522C3940640030260ED7BFF7A6883
:1061B300799F852239748C2522F582E43460F58336
:1061C300E0F53A126AEE7530007531007532247BC2
:1061D300FF7A6879C0126E6A8F23E523B4010E74C7
:1061E3008C2522F582E43460F583E524F0052280D2
:1061F300B17BFF7A68799D126AEEE4F522E522C34A
:10620300940440030260ED7BFF7A6879C4852239E8
:1062130074922522F582E43460F583E0F53A126A3C
:10622300EE7530007531007532247BFF7A6879E7AB
:10623300126E6A8F23E523B4010E74922522F58230
:10624300E43460F583E524F0052280B17BFF7A68AE
:10625300799D126AEEE4F522E522C3940440030219
:1062630060ED7BFF7A6879EB85223974842522F50A
:1062730082E43460F583E0F53A126AEE7530007516
:1062830031007532247BFF7A6879E7126E6A8F23B7
:10629300E523B4010E74842522F582E43460F5838A
:1062A300E524F0052280B17BFF7A68799D126AEEBE
:1062B300E4F522E522C3940440030260ED7BFF7AF8
:1062C30069790785223974882522F582E43460F5DB
:1062D30083E0F53A126AEE753000753100753224A9
:1062E3007BFF7A6879E7126E6A8F23E523B4010E88
:1062F30074882522F582E43460F583E524F00522D1
:1063030080B17BFF7A68799D126AEEE4F522E5227B
:10631300C3940440030260ED7BFF7A6979288522E8
:1063230039749B2522F582E43460F583E0F53A1253
:106333006AEE7530007531007532247BFF7A687917
:10634300E7126E6A8F23E523B4010E749B2522F5B1
:1063530082E43460F583E524F0052280B17BFF7A83
:1063630068799D126AEEE4F522E522C394044003A2
:106373000260ED7BFF7A69794B852239749F252270
:10638300F582E43460F583E0F53A126AEE75300085
:106393007531007532247BFF7A6879E7126E6A8F54
:1063A30023E523B4010E749F2522F582E43460F5BE
:1063B30083E524F0052280B17BFF7A69796E9060D2
:1063C30099E0F539A3E0F53A126AEE7530007531BC
:1063D300007532267BFF7A697992126E6A8F23E504
:1063E30023640160030260EDE52745267003026024
:1063F300ED906099803C7BFF7A697995906097E096
:10640300F539A3E0F53A126AEE753000753100757F
:1064130032267BFF7A697992126E6A8F23E52364B1
:106423000160030260EDE527452670030260ED90ED
:106433006097E526F0A3E527F00260ED7BFF7A691C
:1064430079B39060A3E0F539126AEE7530007531C7
:10645300007532247BFF7A6879E7126E6A8F23E531
:1064630023640160030260EDE52470030260ED9094
:1064730060A3F00260ED7BFF7A6979DC126AEEE4D7
:10648300F523E523C3947F40030260ED127664EFA6
:10649300F522640A6005E522B40D1074002523F586
:1064A30082E43460F583E4F00260EDE522B408246D
:1064B300E523D39400402F7BFF7A6979FF126AEEBC
:1064C300152374002523F582E43460F5837420F0EA
:1064D3001523801274002523F582E43460F583E5E7
:1064E30022F0FF127650052380987BFF7A6A7903A6
:1064F3000265F97BFF7A6A790D126AEEE4F523747B
:10650300B52523F582E43460F583E4F00523E52320
:10651300B408ECE4F523127664EFF522640A60050F
:10652300E522B40D0F74B52523F582E43460F583B9
:10653300E4F08044E522B40824E523D39400402FFB
:106543007BFF7A6979FF126AEE152374B52523F56B
:1065530082E43460F5837420F01523801274B5252A
:1065630023F582E43460F583E522F0FF12765005CB
:1065730023E523C39408409E9060B5E06420600344
:106583000260EDF523E523C3940840030260ED7434
:10659300B52523F582E43460F583E4F0052380E533
:1065A300E4F5250260ED7BFF7A6A7927126AEEE44F
:1065B300F523E52304FF74842523F582E43460F591
:1065C30083E0FD1275EA0523E523C3943F40E3E42A
:1065D300F523E523247FFF74002523F582E434604B
:1065E300F583E0FD1275EA0523E523C3948040E2B9
:1065F3007BFF7A6A793C126AEE0260ED1274B5028F
:1066030060ED7BFF7A0079008B288A29892A12732F
:10661300087F057E001275AE0524E524C394195046
:10662300030260847F2E1276500523E523C3940A68
:1066330050030260817BFF7A0079008B288A2989C5
:066643002A12730880FE1C
:1074B5007BFF7A6A7950126AEE7530007531007576
:1074C500322B7BFF7A697992126E6ABF012DD3E563
:1074D5002C9400E52B940040227BFF7A6A796A128E
:1074E5006AEEAF2CAE2B1275017BFF7A6A797C129E
:0B74F5006AEE7D01AF2CAE2B1273FA83
:017500002268
:02757A008B364E
:10757C00A2AF9200C2AF85A23753A2FE8E838F8238
:10758C0005A28C838D827409127617E53653A2FE00
:10759C0043A22012761953A2DF8537A2A20092AF24
:0175AC00FFDF
:0175AD0022BB
:1075CD00E5D220E0FBC2AF438E2075D2028F8275CB
:0C75DD008300E0FFE4F5D2538EDFD2AF54
:0175E900227F
:1075EA00E5D220E0FBC2AF43D2028F82758300ED61
:0A75FA00F075D25063D250D2AF22D8
:10761700F922C002C004C00612FFF0D006D004D081
:0276270002223D
:03600000027658CD
:0C76580078FFE4F6D8FD7581490260035C
:10728D00BC000BBE0029EF8DF084FFADF022E4CCE5
:10729D00F875F008EF2FFFEE33FEEC33FCEE9DECAE
:1072AD00984005FCEE9DFE0FD5F0E9E4CEFD22EDF4
:1072BD00F8F5F0EE8420D21CFEADF075F008EF2F3E
:1072CD00FFED33FD4007985006D5F0F222C398FD2F
:0572DD000FD5F0EA22CC
:1072E200D083D082F8E4937012740193700DA3A33B
:1072F20093F8740193F5828883E47374029368604F
:06730200EFA3A3A380DF4E
:067308008A838982E47310
:106A8C00E5452439F8E60545227836300702783991
:106A9C00E475F0011273B602730E2000EB7F2ED258
:106AAC00008018EF540F2490D43440D4FF30040BE2
:106ABC00EF24BFB41A0050032461FFE546600215B1
:106ACC00460549E5497002054830070D7836E475EE
:106ADC00F0011273B6EF02735402763A7403D207C4
:106AEC008003E4C207F5458B368A378938E4F546CE
:106AFC00F548F549E54660077F20126AC780F575B1
:106B0C0047FFC201C200C202C203C205C206C208CC
:106B1C00126A95FF700D3007057F00126AD8AF49D5
:106B2C00AE4822B4255FC2D5C204126A95FF24D0A8
:106B3C00B40A00501A75F00A784630D50508B6FF2D
:106B4C000106C6A426F620D5047002D20380D924EF
:106B5C00CFB41A00EF5004C2E5D204026CD8D201B3
:106B6C0080C6D20080C0D20280BCD2D580BAD205F9
:106B7C0080B47F20126AC72002077401B54600401A
:106B8C00F1126A8CFF126AC7026B00D208D206801F
:106B9C0095126A8CFB126A8CFA126A8CF94A4B7049
:106BAC000679A97A6D7BFF20022EE546602A7E00CD
:106BBC008E8275830012732760060EEE654770F0A7
:106BCC00C2D5EBC0E0EAC0E0E9C0E0EE126D1FD028
:106BDC00E0F9D0E0FAD0E0FB12730EFF60AAEBC034
:106BEC00E0EAC0E0E9C0E0126AC7D0E02401F9D0C5
:106BFC00E03400FAD0E0FBE5470460DCD547D980EF
:106C0C00877BFF7A6D791BD202809C791080027988
:106C1C0008C206C2088008D2D5790A8004790AC253
:106C2C00D5E547047002F547E4FAFDFEFF126A8CC5
:106C3C00FC7B08200113126A8CFD7B1030000A12B9
:106C4C006A8CFE126A8CFF7B20EC3382D592D55075
:106C5C0013C3E43000069FFFE49EFEE42001039D75
:106C6C00FDE49CFCE4CBF8C201EC700CCFCECDCC97
:106C7C00E824F8F870F38017C3EF33FFEE33FEED22
:106C8C0033FDEC33FCEB33FB994002FB0FD8E9EB03
:106C9C00300105F8D0E0C448B201C0E00AEC4D4E1A
:106CAC004F78207B0070C2EAB5470040BCC0E012B0
:106CBC006D21D0F0D0E0200104C4C0E0C4B201C00A
:106CCC00F0126AB0D0F0D5F0EB026B001272E26BEE
:106CDC009D536C17586B6E4C6B6A426C1B4F6C233C
:0F6CEC00446C23496B83436C29556C0D466C0D2A
:106CFB00456C0D476DC9506B722D6B762E6B992BB6
:106D0B006B7A236B97206DB22A6B324800006B9124
:106D1B003F3F3F00790AA2D5200314300509B91073
:106D2B00020404B9080104A2D52006025001042074
:106D3B0002689202B546005034C0E07F2030031940
:106D4B007F30A20272067205500F126D78C202C21A
:106D5B0006C205C2087F30800F300503E9C0E01280
:106D6B006AC7300503D0E0F9D0E0B546CC30051743
:106D7B007F30B9100C126AC77F583004077F7880B8
:106D8B0003B90803126AC73002057F2D026AC77F59
:106D9B00202008F87F2B2006F322920280CF286E4A
:106DAB00756C6C2900D201126A8C3001F8C2017823
:106DBB004630D50108F6026B322D50434958126A02
:106DCB008C2403B405004001E4906DC493126AB89F
:0D6DDB00743A126AB8D203754604026C17B0
:106DE800E54230030104F823282430F822782D30B6
:106DF80003027830E475F0011273B602730E60EC8A
:106E0800C5467002154514C546200304FF02767472
:106E1800782D74FFF5F00273C6FF027604E543602F
:106E280006D543037F002220030F127629EF60085E
:106E38000546E5467002054522782D1273AD12739A
:106E48000EFF60E9782DE475F0011273B680DE124A
:106E58006E2FEFC0E0126E21D0E040F380A0D20385
:106E68008002C2038B2D8A2E892FE4F544F542F562
:106E780045F546754300C202C200C201C204126D44
:106E8800F5FF7005AF447E0022B42530126DF5FF82
:106E980024D0B40A00500C75F00AC543A42543F564
:106EA8004380E924CFB41A00EF5002C2E50270CB48
:106EB800D20180D8D20080D4D20480D0EF126E21C3
:106EC8005008126E57EF600E80A9EFC0E0126E2FC7
:106ED800D0E06F609EEF6074126E0680A7126E2F6E
:106EE800EF6069E543700705438003126E2FEF607A
:106EF8001420040E126DE8E475F0011273B6EF1257
:106F08007354D543E62004040542054480BA126E42
:106F180025EFC0E0126E21D0E05004126E06E4FFA7
:106F280020040E126DE8E475F0011273B6EF1273C7
:106F380054EF70DA20040405420544808BE5436071
:106F4800020543126E57126E25EF70C6300304E433
:106F5800126E06E5446003026E8C7EFF7FFF2220DE
:106F6800041174FFFCFDFEFF126DE81273AD12737D
:106F7800930542026E7BD0E080D27900800A7910B6
:106F8800800679088002790AD205E5436002054344
:106F9800E9C0E0126E57EF60DD126E2FBF2D04D2EC
:106FA800028003BF2B09126E57EF60CA126E25D0FC
:106FB800E0B40A028033B40802802EBF3027700282
:106FC8007408C205C0E0126E25D0E0BF78028003C5
:106FD800BF58160543D543028007D54304D2058020
:106FE8000B741080197002740ABF000AEFF8E4FCF1
:106FF800FDFEFF02707EC0E0EF126E06D0E0F9E4FD
:10700800FCFDFEFFE9C0E0ECC0E0EDC0E0EEC0E052
:10701800EFC0E0126E25EFF8D0E0FFD0E0FED0E040
:10702800FDD0E0FCD0F0E8604DB461004007B47BCF
:10703800005002C2E524D0503DFA24F6500724F946
:107048005034240AFAEAB5F000502BCFA9F0A42F47
:10705800FF92D5E9C5F0CEA4A2D53EFE92D5E9C5EA
:10706800F0CDA4A2D53DFD92D5E9C5F0CCA4A2D51A
:0B7078003CFCC205808EE8C0E0200454
:107083002A2005080544300203127385126DE812A5
:1070930073AD054220000B20010DEE8FF0127366D5
:1070A30080091273938004EF127354D0E0126E06BA
:1070B300026E7B200410126DE81273AD0542E545A4
:1070C3008546F012736680E81272E26F45536F864D
:1070D300586EBC4C6EB8426E94486F8A4F6F8E44A4
:1070E3006EE5436F82496F8E556F67466F67456FD5
:0C70F30067476EC02A70B64E00006EC4E5
:10730E00BB010689828A83E0225002E722BBFE027D
:09731E00E32289828A83E49322B0
:10732700BB010CE58229F582E5833AF583E022501B
:1073370006E92582F8E622BBFE06E92582F8E22265
:0D734700E58229F582E5833AF583E493227F
:10735400BB010689828A83F0225002F722BBFE0118
:02736400F32212
:10736600BB010A89828A83F0E5F0A3F0225006F772
:0F73760009A7F01922BBFE06F3E5F009F319226F
:0E738500C3E49FFFE49EFEE49DFDE49CFC2219
:10739300BB010789828A830273E25005E9F802730D
:0A73A300D6BBFE05E9F80273EE22E6
:0973AD00E6FB08E6FA08E6F92205
:1073B600FAE6FB0808E6F925F0F618E6CA3AF622D8
:1073C600FAE6FB0808E625F0F9F618E63AFAF62298
:1076290010090B12766CBF0D027F0A02763AAF0879
:01763900222E
:057674008F08D209227D
:10760400EFC394094005EF940E4003BF2003D380D9
:0376140001C3228D
:0C73D600ECF608EDF608EEF608EFF622E3
:0C73E200ECF0A3EDF0A3EEF0A3EFF0221E
:0C73EE00ECF208EDF208EEF208EFF222DB
:00000001FF
